S0220000687474703A2F2F737265636F72642E736F75726365666F7267652E6E65742F1D
S12300000C9438000C9432190C940F160C945F000C945F000C945F000C945F000C945F0059
S12300200C945F000C94D81B0C945F000C94E41B0C945F000C946A160C94AC160C94B8159E
S12300400C945F000C945F000C945F000C945F000C944A1C0C94121C0C945F000C945F00CE
S12300600C945F000C945F000C945F000C945F0011241FBECFEFD0E1DEBFCDBF14BEA895C7
S123008088E10FB6F89480936000109260000FBE14E0A0E0B1E0EEE0FCE302C005900D92B8
S12300A0A83DB107D9F716E0A8EDB4E001C01D92A23AB107E1F70E94470E0C94061E0C9479
S12300C0000020E030E0D901AC54BF4F0E94E81D802DF901E15CFE4F80832F5F3F4F203AD3
S12300E0310589F720E030E0D901A857BE4F0E94E81D802DF901E85CFE4F80832F5F3F4F52
S12301002530310589F712BC11BC089520E030E0F901E15CFE4F8081D901AC54BF4F082EE5
S12301200E94F51D2F5F3F4F203A310589F712BC11BC089520E030E0D90150960E94E81D2C
S1230140802DF901E152FE4F80832F5F3F4F203A310591F712BC11BC089520E030E0F901FB
S1230160E152FE4F8081D9015096082E0E94F51D2F5F3F4F203A310591F712BC11BC0895E4
S123018020E430E0F901E158FD4F8081D901A05BBE4F082E0E94F51D2F5F3F4F203A31054F
S12301A089F712BC11BC0895A2E0B0E00E94E81D802D90E090931D0180931C0120911C016E
S12301C030911D01A3E0B0E00E94E81D802D90E0982F8827820F931F90931D0180931C013B
S12301E0A4E0B0E00E94E81D802D90E090931F0180931E0120911E0130911F01A5E0B0E0E8
S12302000E94E81D802D90E0982F8827820F931F90931F0180931E01A6E0B0E00E94E81D2B
S1230220802D90E090930101809300012091000130910101A7E0B0E00E94E81D802D90E014
S1230240982F8827820F931F909301018093000180910001909101018072987C9093010148
S123026080930001A1E0B0E00E94E81D802D8093D804A8E0B0E00E94E81D802D809313017F
S1230280A9E5B1E00E94E81D802D8093280180912801843039F481E08093180183E6809387
S12302A0B40503C082E080931801A9E0B0E00E94E81D802D80931201AEE0B0E00E94E81DD8
S12302C0802D80932101ABE0B0E00E94E81D802D80931901ACE0B0E00E94E81D802D809319
S12302E01A01AFE6B1E00E94E81D802D80931B01A2EFB1E00E94E81D802D80934605809151
S12303004605882319F081E080934605ADE0B0E00E94E81D802D26E0829FC001112490936A
S1230320150180931401A1E7B1E00E94E81D802D8093D805A0E7B1E00E94E81D802D80939F
S1230340D6058AE08093050681E080930306A895AFE8B1E00E94E81D802D809329018091B2
S1230360290181FF05C080912901827F809329018091290185FF05C0809129018F728093BE
S12303802901A4EFB1E00E94E81D802D24E1829FC001112490936F0580936E05A5EFB1E059
S12303A00E94E81D802D80936B05A6EFB1E00E94E81D802D80936905A7EFB1E00E94E81D99
S12303C0802D80936805A8EFB1E00E94E81D802D90E0909367058093660520916605309116
S12303E06705A9EFB1E00E94E81D802D90E0982F8827820F931F9093670580936605ABEF40
S1230400B1E00E94E81D802D90E090932B0180932A0120912A0130912B01ACEFB1E00E945F
S1230420E81D802D90E0982F8827820F931F90932B0180932A01ADEFB1E00E94E81D802DCF
S123044090E090932D0180932C0120912C0130912D01AEEFB1E00E94E81D802D90E0982F11
S12304608827820F931F90932D0180932C01AFEFB1E00E94E81D802D90E090932F0180939C
S12304802E0120912E0130912F01A0E0B2E00E94E81D802D90E0982F8827820F931F9093A6
S12304A02F0180932E01ABECB3E00E94E81D802D80934A05ACECB3E00E94E81D802D809354
S12304C04B05ADECB3E00E94E81D802D80934F05AEECB3E00E94E81D802D80933001A895DF
S12304E020E030E0D901A25ABE4F0E94E81D802DF901E15EFC4F8083D901AE58BE4F0E949B
S1230500E81D802DF901EB54FA4F8083D901A458BE4F0E94E81D802D808B2F5F3F4F2A30E8
S1230520310501F7A7E0B2E00E94E81D802D80933301A3E0B2E00E94E81D802D8093340124
S123054020E030E0F901EE51FA4F84E6808BD901A45EBD4F0E94E81D802D80832F5F3F4F35
S12305602031310579F720E030E0D901A759BE4F0E94E81D802DF901ED5DFE4F80832F5F13
S12305803F4F2430310589F720E030E0D901A25DBD4F0E94E81D802DF901EF54FB4F8083EC
S12305A02F5F3F4F2031310589F7ADE6B1E00E94E81D802D80932001A1EFB1E00E94E81DA0
S12305C0802D80934505A0EFB1E00E94E81D802D80932701A6E0B2E00E94E81D802D8093DF
S12305E0220120E030E0D901AA54BC4F0E94E81D802DF901E75DFC4F80832F5F3F4F203194
S1230600310589F7A7ECB3E00E94E81D802D80933601A8ECB3E00E94E81D802D8093370196
S123062012BC11BC089580911C0190911D01A2E0B0E0082E0E94F51D80911C0190911D01A8
S1230640892F9927A3E0B0E0082E0E94F51D80911E0190911F01A4E0B0E0082E0E94F51DB2
S123066080911E0190911F01892F9927A5E0B0E0082E0E94F51D8091000190910101A6E0D3
S1230680B0E0082E0E94F51D8091000190910101892F9927A7E0B0E0082E0E94F51D80911D
S12306A01301A8E0B0E0082E0E94F51D80911201A9E0B0E0082E0E94F51D12BC11BC0895C1
S12306C080E0A1EFB1E0082E0E94F51D8AE0A0EFB1E0082E0E94F51D80914605A2EFB1E0B9
S12306E0082E0E94F51D84E0A9E5B1E0082E0E94F51D85E0ACE0B0E0082E0E94F51D82E3CF
S1230700AFE6B1E0082E0E94F51D24E1A1E7B1E0022E0E94F51D91E0A0E7B1E0092E0E9461
S1230720F51D88ECA4EFB1E0082E0E94F51DA5EFB1E0092E0E94F51DA6EFB1E0022E0E9419
S1230740F51D8AE5A7EFB1E0082E0E94F51D88EEA8EFB1E0082E0E94F51D83E0A9EFB1E0EF
S1230760082E0E94F51D80912A0190912B01ABEFB1E0082E0E94F51D80912A0190912B0164
S1230780892F9927ACEFB1E0082E0E94F51D80912C0190912D01ADEFB1E0082E0E94F51D23
S12307A080912C0190912D01892F9927AEEFB1E0082E0E94F51D80912E0190912F01AFEFE9
S12307C0B1E0082E0E94F51D80912E0190912F01892F9927A0E0B2E0082E0E94F51D8CED1C
S12307E0A7E0B2E0082E0E94F51D86EEA3E0B2E0082E0E94F51D2CE132E088ECD901082EDC
S12308000E94F51D2F5F3F4F82E02C323807A9F782E2AFE8B1E0082E0E94F51D81E0A6E008
S1230820B2E0082E0E94F51D12BC11BC0895CF92DF92EF92FF920F931F93CF93DF93C0E054
S1230840D0E0A5E0B2E00E94E81D202D30E040E050E06E01CC0CDD1C89E393E0C80ED91E8D
S1230860F6016081718180E090E00E94591D24E630E040E050E00E94AB1D79018A01CA011E
S1230880B90124EF31E040E050E00E94591D28EC30E040E050E0E20EF31E041F151FA80199
S12308A097010E94AB1DCA01B9012FEF30E040E050E00E94591D25E030E040E050E00E9410
S12308C0AB1D02E0220F331F441F551F0A95D1F7CA01B90124E630E040E050E00E94AB1D50
S12308E0F601318320832196C732D10509F0A9CFC0E0D0E0A9ECB3E00E94E81D202D30E033
S123090040E050E06E01CC0CDD1C87E893E0C80ED91EF6016081718180E090E00E94591DE2
S123092024E630E040E050E00E94AB1D79018A01CA01B90124EF31E040E050E00E94591DC9
S123094028EC30E040E050E0E20EF31E041F151FA80197010E94AB1DCA01B9012FEF30E069
S123096040E050E00E94591D25E030E040E050E00E94AB1DB2E0220F331F441F551FBA9501
S1230980D1F7CA01B90124E630E040E050E00E94AB1DF601318320832196C732D10509F065
S12309A0A9CFC0E0D0E0AAECB3E00E94E81D202D30E040E050E06E01CC0CDD1C85ED93E0C9
S12309C0C80ED91EF6016081718180E090E00E94591D24E630E040E050E00E94AB1D790146
S12309E08A01CA01B90124EF31E040E050E00E94591D28EC30E040E050E0E20EF31E041FBF
S1230A00151FA80197010E94AB1DCA01B9012FEF30E040E050E00E94591D25E030E040E0A3
S1230A2050E00E94AB1DF2E0220F331F441F551FFA95D1F7CA01B90124E630E040E050E0A6
S1230A400E94AB1DF601318320832196C732D10509F0A9CFC0E0D0E0A4E0B2E00E94E81DD6
S1230A60202D30E040E050E06E01CC0CDD1C83E294E0C80ED91EF6016081718180E090E045
S1230A800E94591D24E630E040E050E00E94AB1D79018A01CA01B90124EF31E040E050E068
S1230AA00E94591D28EC30E040E050E0E20EF31E041F151FA80197010E94AB1DCA01B9011E
S1230AC02FEF30E040E050E00E94591D25E030E040E050E00E94AB1D72E0220F331F441F75
S1230AE0551F7A95D1F7CA01B90124E630E040E050E00E94AB1DF601318320832196C73250
S1230B00D10509F0A9CFDF91CF911F910F91FF90EF90DF90CF900895EAE7F0E0108280E25C
S1230B2080937C00089809980A980B980E980F9880E880BF87EE808308950F931F93CF93DD
S1230B40DF93282F30E0F901EE0FFF1FEE5FFE4F0081118143E0033F140718F0E2E3F0E0D9
S1230B604CC053E00F3D150718F0EAE0F0E045C0C0E0D0E087E290E0A901489F9001499FF0
S1230B80300D589F300D1124D901AC0FBD1FAA0FBB1FA75CBC4F8D919C9111978017910777
S1230BA030F5FE013197E20FF31FEE0FFF1FE75CFC4F20813181608171814D915C91FE01A9
S1230BC0EE0FFF1FEE0FFF1FEC0FFD1F3596201B310BC901880F991F880F991F641B750B1B
S1230BE0820F931F0E94841DE60FF71F06C02196C732D10549F6E8ECF0E0CF01DF91CF9191
S1230C001F910F9108950F931F93CF93DF93AC01E0E0F0E0EF01CC0FDD1FDE01AF58BB4FC7
S1230C208D919C91119748175907C0F56D917C913197EE0FFF1FDF01AF58BB4F8D919C911F
S1230C401197681B790B8D919C91C757DB4F28813981E757FB4F00811181481B590B84E61F
S1230C6090E0DC014A9FC0014B9F900D5A9F900D11240E94841D201B310B0190F081E02D5E
S1230C80629FC001639F900D729F900D112464E670E00E94841D6E0F7F1F09C03196EA306A
S1230CA0F10509F0B7CF60919D0470919E04CB01DF91CF911F910F910895809100019091CA
S1230CC0010197FD2BC02091390530913A0580911C0190911D01C29682179307C8F020913F
S1230CE0390530913A0580911C0190911D0149978217930768F02091390530913A058091DA
S1230D001C0190911D018B5490408217930730F48091480590914905816005C0809148059C
S1230D20909149058E7F9093490580934805809100019091010193FF1DC0339906C080911B
S1230D404E058F5F80934E0502C010924E0580914E05853130F08091480590914905826048
S1230D6005C080914805909149058D7F909349058093480590915B0580913001891730F479
S1230D808091480590914905886005C08091480590914905877F9093490580934805209180
S1230DA0E8043091E9048091340190E08217930734F48091480590914905806105C0809100
S1230DC04805909149058F7E90934905809348058091DA049091DB048E37910534F08091F6
S1230DE0480590914905806217C08091DA049091DB048A3691055CF080914805909149051C
S1230E008062909349058093480521E00AC080914805909149058F7D9093490580934805A6
S1230E2020E08091DE049091DF048C39910534F08091480590914905806405C08091480564
S1230E40909149058F7B90934905809348058091DA049091DB048B3A910534F08091480578
S1230E6090914905806805C080914805909149058F779093490580934805222321F082E3F3
S1230E80809335050895109235050895809100019091010193FFF3C0339906C080914E057B
S1230EA08F5F80934E0502C010924E0580914E05833328F12091390530913A0580912E01C1
S1230EC090912F018217930730F48091E0059091E105986005C08091E0059091E105977F99
S1230EE09093E1058093E00580914B0590E090934D0580934C0584E380934E05A6C08091FF
S1230F004C0590914D05892B09F49FC080914A05823069F1833030F4882359F0813009F018
S1230F2082C00AC0833009F43DC0843009F07BC065C010924B0589C02091390530913A05BD
S1230F4080912E0190912F018217930730F48091E0059091E105986005C08091E0059091D4
S1230F60E105977F9093E1058093E00539C02091390530913A0580912E0190912F0182175E
S1230F80930730F48091E0059091E105986005C08091E0059091E105977F9093E1058093A6
S1230FA0E00553C08091E0059091E105977F9093E1058093E00590915B05809130018917BE
S1230FC030F48091B0059091B105886005C08091B0059091B105877F9093B1058093B0055B
S1230FE08091DA049091DB0480934B0580914B058B3F58F18AE080934B0527C08091E0057D
S12310009091E105977F9093E1058093E00590915B0580913001891778F48091B0059091F8
S1231020B10588600EC08091E0059091E105977F9093E1058093E0058091B0059091B1058F
S1231040877F9093B1058093B00580914A05853041F590915B0580913001891730F4809102
S1231060B0059091B105886005C08091B0059091B105877F9093B1058093B0050895809141
S1231080E0059091E105977F9093E1058093E0058091B0059091B105877F9093B1058093BA
S12310A0B0050895A89582E50E949F1C83E10E949F1C8091390590913A05892F99270E944F
S12310C09F1C8091390590913A050E949F1C8091DE049091DF040E949F1C8091DA049091E1
S12310E0DB040E949F1C8091E6049091E7040E949F1C8091E8049091E9040E949F1C8091D3
S1231100DC049091DD040E949F1C8091E2049091E3040E949F1C8091DB059091DC05969512
S123112087950E949F1C80913E050E949F1C80913D050E949F1C2091E0053091E105809183
S1231140B0059091B105E3E096958795EA95E1F78170232F3327822B0E949F1C8091E00501
S12311609091E1050E949F1C809113010E949F1C80915B050E949F1C8091E0049091E104BC
S12311800E949F1C8091B2059091B305969587950E949F1C2091580530E0220F331FF9010E
S12311A0E651FB4F80819181892F990F990B93E0220F331F9A95E1F7822B0E949F1CE0911B
S12311C05805F0E0EE0FFF1FE651FB4F808191810E949F1C8DEA0E949F1C809158058F5FA2
S12311E080935805883010F0109258050895CF92DF92FF920F931F93CF93DF93A89588E1F6
S12312000FB6F89480936000109260000FBE0E94EB1C882309F41DC50E947C1C909357054B
S1231220809356058236910509F4E3C283369105E8F58035910509F456C381359105E8F497
S12312408534910509F4CDC08634910568F48932910509F451C48134910509F489C0883257
S1231260910509F0F4C425C48634910509F442C18D34910509F0EBC4B9C18735910509F422
S1231280A9C38835910548F48235910509F4A7C38335910509F0DBC481C48835910509F420
S12312A0D6C38136910509F0D2C43DC08936910509F4CAC28A369105C8F48536910509F47A
S12312C008C28636910548F48336910509F494C28436910509F0BBC4BCC48636910509F479
S12312E0E7C08736910509F0B2C4D5C28037910509F4FEC28137910548F48D36910509F400
S123130034C18F36910509F0A2C4B9C38937910509F415C48A37910509F471C28837910596
S123132009F095C46CC281E60E949F1C80EA0E949F1C10925705109256050EC0E15CFE4F4B
S123134080810E949F1C809156059091570501969093570580935605E0915605F091570515
S1231360E03AF10558F382E30E94F01B8EE96FC41092570510925605C0E0D0E00E94EB1C5E
S1231380882341F1C0915605D0915705C03AD10589F40E947C1C90935705809356058E3BC6
S12313A0910519F4C6E1DAEF15C0809156050E949F1CFBCF0E947C1CC15CDE4F888380910E
S12313C056059091570501969093570580935605C0E0D0E021964AEFC030D40708F039C4AD
S12313E0CDCFC0E0D0E00E94EB1C882309F459C00E947C1C8A3B910509F02BC488E10FB6E8
S1231400F89480936000109260000FBE10925705109256053EC0885B0E949F1C8DEF0E94A3
S12314209F1C20915605309157058AEF90E0289FE001299FD00D389FD00D112407C0DE01FF
S12314400E94E81D802D0E949F1C219620915605309157052F5F3F4F8AEF90E0AC01249F82
S1231460C001259F900D349F900D112421503040C817D90720F3822F885B80950E949F1CE8
S123148080915605909157050196909357058093560580915605909157058430910508F4AC
S12314A0BACF21965AEFC030D50708F0D2C39BCF86E60E949F1C80EA0E949F1C109257054E
S12314C0109256050EC0E152FE4F80810E949F1C809156059091570501969093570580934D
S12314E05605E0915605F0915705E03AF10558F389E9ADC3109257051092560500E010E0DC
S12315000E94EB1C882349F1C0915605D0915705C03AD10591F40E947C1C909357058093AF
S12315205605893B910519F406E11AEF16C0E0915405F0915505099510C00E947C1CC152BF
S1231540DE4F888380915605909157050196909357058093560500E010E00F5F1F4F8AEFBD
S12315600030180708F075C3CBCF8DE60E949F1C89E00E949F1C80911C0190911D010E94A9
S12315809F1C80911C0190911D01892F99270E949F1C80911E0190911F010E949F1C80916B
S12315A01E0190911F01892F99270E949F1C80910001909101010E949F1C8091000190912D
S12315C00101892F99270E949F1C809113010E949F1C809112010E949F1CAAE0B0E00E9471
S12315E0E81D802D0E949F1C82E931C31092570510925605C0E0D0E00E94EB1C8A3008F4CF
S123160061C00E947C1C90931D0180931C0100911C0110911D010E947C1C982F8827800F4E
S1231620911F90931D0180931C010E947C1C90931F0180931E0100911E0110911F010E94C3
S12316407C1C982F8827800F911F90931F0180931E010E947C1C90930101809300010091C0
S12316600001109101010E947C1C982F8827800F911F90930101809300010E947C1C80934D
S123168013010E947C1C809312010E947C1CAAE0B0E0082E0E94F51D0E94D71B0E947C1CC6
S12316A0823B910551F40E941303E0915405F09155050995CFE6DAEF05C0E0915405F09105
S12316C05505099521964AEFC030D40708F0C1C293CF85E60E949F1C83E10E949F1C10924B
S12316E05705109256050EC0E15EFC4F80810E949F1C8091560590915705019690935705D8
S123170080935605E0915605F0915705EA30F10558F3809119010E949F1C80911A010E94FD
S12317209F1C83E00E94F11B809123010E949F1C809124010E949F1C809125010E949F1C20
S1231740809126010E949F1C809114019091150166E070E00E94841DCB010E949F1C809180
S123176020010E949F1CAEE6B1E00E94E81D802D0E949F1C8AE90E949F1C8CE60E949F1C72
S123178084E10E949F1C10925705109256050EC0EB54FA4F80810E949F1C80915605909147
S12317A0570501969093570580935605E0915605F0915705EA30F10558F3109257051092A1
S12317C056050EC0EB54FA4F80890E949F1C80915605909157050196909357058093560581
S12317E0E0915605F0915705EA30F10558F383E92EC20E9486002DC20E94AD002AC20E9491
S1231800520827C20E947C1CC82FD0E00E947C1CC817D90709F01DC20E947C1C8C019093E5
S12318205705809356050E947C1C0817190709F010C20E947C1C8639910509F00AC2809131
S12318405605C15CDE4F4DC00E94EB1C8530D0F6FBCF0E947C1CC82FD0E00E947C1CC817EA
S1231860D90709F0F6C10E947C1C8C0190935705809356050E947C1C0817190709F0E9C104
S12318800E947C1C8839910509F0E3C180915605C152DE4F26C00E94EB1C8530D0F6FBCF96
S12318A00E947C1CC82FD0E00E947C1CC817D90709F0CFC10E947C1C8C0190935705809368
S12318C056050E947C1C0817190709F0C2C10E947C1C8F3A910509F0BCC180915605C15820
S12318E0DD4F8883B6C10E94EB1C8530C8F6FBCFC0E0D0E00E94EB1C823080F10E947C1CFA
S12319000E947C1C8F38910509F0A3C110925705109256051CC0E158FD4F108180E70E94D9
S12319209F1C82E00E949F1C809156050E949F1C812F0E949F1C8FE80E949F1C8091560513
S12319409091570501969093570580935605E0915605F0915705E03AF105E8F221965AEFEF
S1231960C030D50709F475C1C5CF0E947C1C8C010E947C1CD82FCC27C00FD11F0E947C1CDC
S12319808C0190935705809356050E947C1C0817190709F05EC10E947C1C883A9105A9F409
S12319A0DE010E94F01DE0708091560590915705E82BF92BF0935705E0935605DE010F0189
S12319C00E94011E12BC11BC44C1E0915405F091550509950E94EB1C853038F6FBCFCC2419
S12319E0DD240E94EB1C833040F10E947C1CEC010E947C1C8C010E947C1C8D3A910509F0D7
S1231A0028C1102F00270C0F1D1FD8010E94E81DF02C84E50E949F1C83E00E949F1C8F2D3E
S1231A200E949F1C802F0E949F1C012F1127802F0E949F1C8BEA0E949F1C0894C11CD11C8D
S1231A4080E0C8168AEFD80609F403C1CACFC0E0D0E00E94EB1C882359F00E947C1C873AAB
S1231A60910509F0F6C0E0915405F0915505099521964AEFC030D40709F4EBC0EACFC0E01E
S1231A80D0E00E94EB1C882369F00E947C1C8039910509F0DEC00E94C000E0915405F09118
S1231AA05505099521965AEFC030D50709F4D1C0E8CFC0E0D0E00E94EB1C8823B1F00E9432
S1231AC07C1C873D910509F0C4C08091DC049091DD04ADE6B1E0082E0E94F51D12BC11BCF7
S1231AE0E0915405F0915505099521968AEFC030D80709F4AEC0DFCFC0E0D0E00E94EB1C8E
S1231B008823B1F00E947C1C863D910509F0A1C08091DC049091DD04AEE6B1E0082E0E9498
S1231B20F51D12BC11BCE0915405F0915505099521964AEFC030D40709F48BC0DFCFC0E060
S1231B40D0E00E94EB1C823010F10E947C1C892B09F07FC00E947C1C86389105C1F489E79C
S1231B600E949F1C85E00E949F1C88EC0E949F1C80E20E949F1C89E00E949F1C8DE50E94D8
S1231B809F1C80E20E949F1C86E80E949F1C21965AEFC030D50709F45CC0D3CFC0E0D0E025
S1231BA00E94EB1C823008F44CC00E947C1C892B09F047C00E947C1C8C3A910509F049C038
S1231BC083E50E949F1C88E00E949F1C80914105909142050E949F1C80914105909142059C
S1231BE0892F99270E949F1C8091DE059091DF050E949F1C8091DE059091DF05892F992745
S1231C000E949F1C8091D9059091DA050E949F1C8091D9059091DA05892F99270E949F1C53
S1231C2080910D0690910E060E949F1C80910D0690910E06892F99270E949F1C8CEA0E94A4
S1231C409F1C21968AEFC030D80719F0A9CF0E949F1CA895DF91CF911F910F91FF90DF908D
S1231C60CF90089520E931E0D9010E94E81D802D20553140F901E158FD4F80832F5A3E4F9E
S1231C8081E0203F380781F712BC11BC0895CF93DF9314BEA89588E10FB6F8948093600081
S1231CA0109260000FBE8FEF9FEF909301018093000180910001909101018072987C9093AE
S1231CC00101809300011092E1051092E005209A219A259A249A289A299A2D9A2C9A229A1B
S1231CE0239A279A2A9A2B982F9852985A9A5398549A559A569A3A98429A3B98439A39984F
S1231D00419A3C983D983E980D980C980E94F31BAAE5B1E00E94E81D802D809347050E94F7
S1231D2086150E948C050E9417042A9A2B98A7E0B0E00E94E81D802D12BC11BC85FF9BC0A8
S1231D4080910001909101019F7D90930101809300010E9413030E9460030E94AD000E9447
S1231D6086000E94C00086E0AAE0B0E0082E0E94F51D89E1ABE0B0E0082E0E94F51D8EE12F
S1231D80ACE0B0E0082E0E94F51DAEE0B0E0082E0E94F51D20E030E0F901E15EFC4F80819C
S1231DA0D901A25ABE4F082E0E94F51D2F5F3F4F2A30310589F780912301A9E6B1E0082E9B
S1231DC00E94F51D80912401AAE6B1E0082E0E94F51D80912501ABE6B1E0082E0E94F51DC7
S1231DE080912601ACE6B1E0082E0E94F51D20E030E0F901EB54FA4F8081D901AE58BE4F1A
S1231E00082E0E94F51D2F5F3F4F2A30310589F720E030E0F901EB54FA4F8089D901A45837
S1231E20BE4F082E0E94F51D2F5F3F4F2A30310589F78091D805A1E7B1E0082E0E94F51D8A
S1231E40809114019091150166E070E00E94841DADE0B0E0062E0E94F51D84E1ADE6B1E0BA
S1231E60082E0E94F51D81EEAEE6B1E0082E0E94F51D12BC11BC0E94D4000E949A000E9407
S1231E806100809100019091010185FD07C080916F008B7F80936F00289A299A809122019A
S1231EA0882311F480EC01C080E4809335011092D90480911401909115018D5D954030F0D9
S1231EC08CED95E090931501809314011092360586B3866086BB78948AEA0E949F1C80E035
S1231EE00E949F1C85E50E949F1C80916E00836080936E002A9A78942B9AA89580913905B6
S1231F0090913A058E36910520F180913605882301F58091E0059091E1059F7E9093E105E2
S1231F208093E0058091E0059091E10580629093E1058093E0058FE0809336052A9A809133
S1231F40E0059091E10590629093E1058093E0053BC0809136058823B9F180913905909192
S1231F603A058536910580F580916F008D7F80936F00809170008C7F8093700080916F00BB
S1231F808B7F80936F008091E0059091E1058F7D9093E1058093E0058091E0059091E105AA
S1231FA0877F9093E1058093E005289A299A109236058091E0059091E1059F7D9093E10592
S1231FC08093E005109234058091390590913A058558934038F0809136058F3019F48FEF0D
S1231FE080933605809136058F30E8F080913405843081F480916F00856080936F00809141
S12320006F00826080936F008091700083608093700005C080913405853008F000005C9A50
S12320202A9A2B9A07C010923405289A299A5C985D9A2D984091390550913A0520911E013D
S123204030911F01809100019091010180709074822B932B4817590788F48091E0059091B5
S1232060E10597FD0BC08091E0059091E1059F7B9093E1058093E0052C9A0AC08091E00579
S12320809091E10590649093E1058093E0052C98F89480914105909142058A5A9A4AC1F0B8
S12320A080914105909142058555954589F078948091E0059091E10580649093E105809327
S12320C0E00588EE93E090933201809331010AC078948091E0059091E1058F7B9093E105AD
S12320E08093E005F89480914305909144058A5A9A4AC1F0809143059091440585559545A5
S123210089F078948091E0059091E10580689093E1058093E00588EE93E0909332018093FE
S123212031010AC078948091E0059091E1058F779093E1058093E0058091310190913201F8
S12321400B9758F02F9A80913101909132010197909332018093310101C02F988091D90488
S1232160833009F4E6C0843020F4813009F09BC0B3C1853009F4EAC1853008F42BC1863014
S123218021F0873009F061C220C280913705909138058D52914008F45BC2E091D904F0E0E3
S12321A080917800909179008C7F65E070E00E94841DEE0FFF1FEA5EFA4F71836083809181
S12321C0D904C82FD0E0E091D904F0E0EE0FFF1FE652FB4F80819181E091D904F0E0EE0F8E
S12321E0FF1FEA5EFA4F20813181880F991F880F991F820F931F880F991F6AE070E00E946D
S1232200841DCC0FDD1FC652DB4F7983688310923805109237058091D9048F5F8093D90490
S12322208091D904806480937C000E94F7088091E6049091E7048035910564F42091140128
S123224030911501C901880F991F820F931F9695879504C0809114019091150190931701A4
S12322608093160180914C0590914D05892B49F080914C0590914D05019790934D05809379
S12322804C0580913D0190913E01892B09F4A0C080913D0190913E01019790933E0180936D
S12322A03D012A9A95C080913705909138058D52914008F4CDC1A091D904B0E0E091D904F2
S12322C0F0E0EE0FFF1FE652FB4F2081318180917800909179009695879596958795280F52
S12322E0391F36952795AA0FBB1FA652BB4F11963C932E931092380510923705A895809124
S12323004C0590914D05892B49F080914C0590914D05019790934D0580934C058091D904D4
S12323208F5F8093D9048091D904806480937C008FC180913705909138058D52914008F4B3
S123234087C1E091D904F0E080917800909179009695879596958795EE0FFF1FEA5EFA4FB6
S1232360918380838091D904C82FD0E0E091D904F0E0EE0FFF1FE652FB4F80819181E0916E
S1232380D904F0E0EE0FFF1FEA5EFA4F20813181880F991F880F991F820F931F65E070E017
S12323A00E94841DCC0FDD1FC652DB4F7983688310923805109237058091D9048F5F80932A
S12323C0D9048091D904806480937C000E94F708A8953EC180913705909138058D52914083
S12323E008F436C180912201882339F1E091D904F0E0809178009091790073E09695879502
S12324007A95E1F790E0EE0FFF1FEA5EFA4F91838083A091D904B0E0E091D904F0E0EE0FE5
S1232420FF1FEA5EFA4F80819181AA0FBB1FA652BB4F11969C938E9340C0E091D904F0E02C
S123244080917800909179009695879596958795EE0FFF1FEA5EFA4F918380838091D90416
S1232460C82FD0E0E091D904F0E0EE0FFF1FE652FB4F40815181E091D904F0E0EE0FFF1F2A
S1232480EA5EFA4F20813181C901880F991F820F931F9A0163E0220F331F6A95E1F7241B81
S12324A0350B820F931F6AE070E00E94841DCC0FDD1FC652DB4F7983688310923805109237
S12324C037058091D9048F5F8093D9048091D904806480937C007CCF809137059091380599
S12324E08D52914008F4B4C0E091D904F0E080917800909179009695879596958795EE0FEC
S1232500FF1FEA5EFA4F918380838091D904C82FD0E0E091D904F0E0EE0FFF1FE652FB4FA1
S123252080819181E091D904F0E0EE0FFF1FEA5EFA4F20813181880F991F880F991F820F38
S1232540931F880F991F6AE070E02ACF80913705909138058D52914008F47AC0E091D90404
S1232560F0E080917800909179009695879596958795EE0FFF1FEA5EFA4F91838083E091A2
S1232580D904F0E0EE0FFF1FEA5EFA4F2081318184E190E0AC01249FC001259F900D349F51
S12325A0900D11240E9403069093E5048093E4048091E4049091E50462E070E00E94981DA7
S12325C07093E5046093E404F3CE80913705909138058D529140E0F1E091D904F0E0809114
S12325E0780090917900969587959695879590E0EE0FFF1FEA5EFA4F91838083A091D904F6
S1232600B0E0E091D904F0E0EE0FFF1FE652FB4F20813181E091D904F0E0EE0FFF1FEA5E97
S1232620FA4F80819181820F931F96958795AA0FBB1FA652BB4F11969C938E931092380545
S1232640109237051092D904BCCE81E08093D9048091370590913805019690933805809389
S123266037058091390590913A058F55914008F457C0809104068F5F809304069091040652
S123268080910506981708F44EC0109204068091E8049091E904E0911306FF27E7FDF09591
S12326A0EE51FA4F208130E08217930734F48091020690910306890F17C08091E8049091B2
S12326C0E904E0911306FF27E7FDF095EE51FA4F208130E0821793074CF08091020682307D
S12326E02CF08091020681508093020680910206E0911306FF27E7FDF095EE51FA4F208952
S1232700992787FD909530E02817390764F4E0911306FF27E7FDF095EE51FA4F808901C0FA
S123272081E0809302068091390590913A058739910508F461C02091DC043091DD048091B3
S1232740200190E04996281739070CF055C080916C0590916D05019690936D0580936C05B0
S123276020916C0530916D0580916E0590916F052817390708F442C010926D0510926C0543
S12327802091390530913A0580916605909167052817390730F490916A0580916B05890FF1
S12327A015C02091390530913A05809166059091670549968217930758F490916A05809149
S12327C06905891728F480916A05815080936A0590916A0580916805891718F480916805C0
S12327E008C090916A0580916905981738F48091690580936A0502C010926A058091D80462
S123280082FF1BC08091390590913A05805D9740A0F42091DC043091DD048091200190E08C
S12328200596281739074CF481E0809352058091E0059091E105916007C0109252058091B0
S1232840E0059091E1059E7F9093E1058093E005809100019091010192FF27C020913905CE
S123286030913A0580912A0190912B0182179307E0F42091390530913A0580912C01909176
S12328802D012817390788F42091DC043091DD048091200190E005962817390734F48091E3
S12328A0E0059091E105946005C08091E0059091E1059B7F9093E1058093E00580915B05E6
S12328C090E09093EB048093EA0480914E0590E09093ED048093EC048091300190E09093B1
S12328E0EF048093EE0480914C0590914D059093F1048093F0048091DA049091DB049093D6
S1232900F3048093F204809100019091010193FFEAC0339906C080914E058F5F80934E05F8
S123292002C010924E0580914E05833328F12091390530913A0580912E0190912F01821790
S1232940930730F48091E0059091E105986005C08091E0059091E105977F9093E1058093CC
S1232960E00580914B0590E090934D0580934C0584E380934E05A6C080914C0590914D05BC
S1232980892B09F48DC080914A05823069F1833030F4882359F0813009F082C00AC0833095
S12329A009F43DC0843009F07BC065C010924B0589C02091390530913A0580912E01909181
S12329C02F018217930730F48091E0059091E105986005C08091E0059091E105977F90937C
S12329E0E1058093E00539C02091390530913A0580912E0190912F018217930730F4809114
S1232A00E0059091E105986005C08091E0059091E105977F9093E1058093E00553C08091D1
S1232A20E0059091E105977F9093E1058093E00590915B0580913001891730F48091B00542
S1232A409091B105886005C08091B0059091B105877F9093B1058093B0058091DA0490919A
S1232A60DB0480934B0580914B058B3F58F18AE080934B0527C08091E0059091E105977FD5
S1232A809093E1058093E00590915B0580913001891778F48091B0059091B10588600EC00F
S1232AA08091E0059091E105977F9093E1058093E0058091B0059091B105877F9093B10582
S1232AC08093B00580914A05853009F014CA90915B0580913001891778F48091B005909188
S1232AE0B10588600EC08091E0059091E105977F9093E1058093E0058091B0059091B105B5
S1232B00877F9093B1058093B005F5C9109280008AEA90E0909389008093880090938B0051
S1232B2080938A0083E08093810080916F00876080936F0080E09AEF9093850080938400EC
S1232B4052985A9A209A219A289A299A80914705813021F480916900836003C080916900DC
S1232B6082608093690081E080931406E89A08951F920F920FB60F9211248F939F93F89479
S1232B80809114068F5F8093140680911406882309F43DC08091E0059091E105906190930A
S1232BA0E1058093E005109236058091E0059091E1059F7D9093E1058093E00580916F00BC
S1232BC08B7F80936F0080916F008D7F80936F00809170008C7F809370005C98289A299ACF
S1232BE08091E0059091E1058F7D9093E1058093E0058091E0059091E105877F9093E105BB
S1232C008093E0052A9810923A051092390578949F918F910F900FBE0F901F9018951F92C1
S1232C200F920FB60F9211240F900FBE0F901F90189580910F06882319F180911806882338
S1232C4089F428988091410590914205880F991F90934205809341058091410590914205A3
S1232C60816007C029988091410590914205880F991F909342058093410510920F0621C07E
S1232C8080910706882389F4289A8091430590914405880F991F909344058093430580913E
S1232CA0430590914405816007C0299A8091430590914405880F991F90934405809343051A
S1232CC02D9A8091E0059091E10593FF02C0289A299A08951F920F920FB60F9211242F9307
S1232CE03F934F935F936F937F938F939F93AF93BF93EF93FF93F89491E090930F068091D4
S1232D005905882319F410920F0614C080915905833051F480910706882319F01092180615
S1232D2007C09093180604C080910706809318060E9419167894FF91EF91BF91AF919F91C7
S1232D408F917F916F915F914F913F912F910F900FBE0F901F9018951F920F920FB60F92C0
S1232D6011242F933F934F935F936F937F938F939F93AF93BF93EF93FF930E9419167894C5
S1232D80FF91EF91BF91AF919F918F917F916F915F914F913F912F910F900FBE0F901F9015
S1232DA01895CF93DF93EC0110921006809110066AE00E94781D80930806809108068A3047
S1232DC01CF089E0809308068091390590913A05885E934008F07DC08091390590913A050D
S1232DE064E670E00E94841D655060930C0680910C0618161CF010920C0607C080910C063D
S1232E0085308CF085E080930C06E0910C06FF27E7FDF095E85CFE4F808190E09093B30504
S1232E208093B20544C0E0910C06FF27E7FDF095E75CFE4F6081E0910C06FF27E7FDF0952B
S1232E40E85CFE4F4081E0910C06FF27E7FDF095E85CFE4F808190E09093B3058093B20563
S1232E60E091B205F091B3058091390590913A0520910C0670E0641B7109845F91404CE949
S1232E80240290011124820F931FAC01649FC001659F900D749F900D112464E670E00E94CC
S1232EA0841DE60FF71FF093B305E093B205109206068FEF8093130680910806992787FD42
S1232EC0909544E0880F991F4A95E1F780933D058AC08091390590913A058B5B9C42E8F0B5
S1232EE088EC8093060684E18093130680910806909113068295807F890F80933D05E091DD
S1232F003D05F0E0E15CFE4F808190E0880F991F9093B3058093B20566C080913905909116
S1232F203A05885E934062E370E00E94841D60930606809106066AE00E94781D80931306F4
S1232F4080910806909113068295807F890F80933D05E0913D05F0E0E15CFE4F808190E093
S1232F60880F991F9093B3058093B2058091130687FD39C0809113068F30ACF5E0913D0575
S1232F80F0E0E05CFE4F8081E0913D05F0E0E15CFE4F6081E091B205F091B30520910606C7
S1232FA040911306861B880F992787FD909530E06AE04602A0011124241B350BAC01429FFD
S1232FC0C001439F900D529F900D11246AE070E00E94981D772767FD70956E0F7F1F7093D4
S1232FE0B3056093B2058091B0059091B10583FF64C080914F05823089F48091B2059091AB
S1233000B3058B3A910538F08091B2059091B3058659904028C084E190E025C080914F051A
S1233020813049F48091090690E083709070892B09F043C00BC080914F058823C9F48091C2
S1233040090690E083709070892BB9F18091B2059091B3058739910580F18091B20590914B
S1233060B3058C5890409093B3058093B20525C080914F05833041F48091090690E0837086
S12330809070892BD1F010C080914F05843041F48091090690E083709070892B71F404C039
S12330A080914F05853049F48091E0059091E10598609093E1058093E0058091390590914F
S12330C03A05855F914010F46AEB66C08091390590913A058952934210F06DE05DC080919F
S12330E0390590913A0585569941B0F08091390590913A05845699416AE070E00E94841D99
S1233100CB01880F991F880F991F860F971F64E670E00E94841D40C08091390590913A056A
S1233120815A9F40B0F08091390590913A05805A9F406AE070E00E94841DCB01A3E0880F06
S1233140991FAA95E1F764E670E00E94841D645123C08091390590913A05855F914010F4BF
S123316060E01AC08091390590913A05845F91406AE070E00E94841DCB019B01F3E0220F85
S1233180331FFA95E1F7880F991F820F931F64E670E00E94841D67532091B2053091B30568
S12331A0862F992787FD9095820F931F97FF06C08091B2059091B30561E0681B80915B0578
S12331C084568B300CF08AE08C3E0CF48CEE992787FD909540916405509165059A01220FF2
S12331E0331F240F351F820F931F262F332727FD3095820F931F64E070E00E94981DAB013D
S123320070936505609364056091B2057091B3052091120160587040620F711D640F751F4E
S123322080E090E02091B2053091B305240F351F3093DC052093DB0520913B0530913C0528
S12332402C0F3D1F40E050E00E94591D28E037E040E050E00E94CD1DC21BD30BCE01DF9176
S1233260CF9108951F920F920FB60F9211241F932F933F934F935F936F937F938F939F93DE
S1233280AF93BF93EF93FF938091DE048F5F8093DE0480918400909185008436910508F425
S12332A072C2809134058F5F8093340580911406882349F08CED9FEF9093120680931106D7
S12332C0109214065FC0E0918400F091850020911106309112068091110690911206369547
S12332E027956AE070E00E94841D261B370BE217F30720F481E08093170645C280913905C0
S123330090913A05845F914010F18091390590913A0584599141D8F480918400909185002F
S12333202091110630911206821B930B90933C0580933B0580913B0590913C0564E070E0AF
S12333400E94981D70933C0560933B0504C010923C0510923B0580913B0590913C05181631
S1233360190624F410923C0510923B05809184009091850090931206809311061092850086
S123338010928400289B02C0299909C080910A0690910B061816190614F40E941916809169
S12333A009068F5F8093090680911106909112069093DF058093DE058091390590913A05DD
S12333C02091DE053091DF051091810040E050E060E070E489E191E00E94CD1DCA01B901BE
S12333E02EE130E040E050E00E94591D20EC129F9001112420503240442737FD4095542FE6
S12334000E94AB1D30933A05209339058091600590916105909363058093620580915E05D5
S123342090915F05909361058093600580915C0590915D0590935F0580935E0580913905C1
S123344090913A0590935D0580935C058091390590913A0589559B41E0F480913905909162
S12334603A0589559240A8F080915B0540915C0550915D05209162053091630590E0821B8D
S1233480930B840F951F9695879596958795855B01C084E680935B058091390590913A0588
S12334A08C52914020F580918100833001F5809117068823E1F484E080938100109285003C
S12334C0109284008091110690911206969587959695879590931206809311068091DE057A
S12334E09091DF0596958795969587952AC08091390590913A058752924038F18091810036
S1233500843019F5809117068823F9F483E080938100109285001092840080911106909192
S12335201206880F991F880F991F90931206809311068091DE059091DF05880F991F880F8D
S1233540991F9093DF058093DE058091DE059091DF050E94D11690930E0680930D068091C2
S1233560390590913A05825C914018F488EE93E009C08091390590913A058C5D954038F4A3
S123358088EC90E0909316068093150604C01092160610921506F8948091170680930706BD
S12335A01092170680910D0690910E0620911401309115014091150650911606821B930B2E
S12335C0841B950B90930B0680930A0680910D0690910E0690938B0080938A0080910A068C
S12335E090910B0697FF1DC020910A0630910B068091DE059091DF05309521953F4F969562
S123360087958217930768F48091DE059091DF0596958795909581959F4F90930B0680934B
S12336200A064091390550913A0520911C0130911D01809100019091010180709078822BC0
S1233640932B4817590708F086C08091E0059091E10593FD80C080910D0690910E064091B4
S1233660140150911501209115063091160684569040240F351F28173907F0F480910A06DC
S123368090910B0690938900809388008091E0059091E1059F779093E1058093E005809188
S12336A0E0059091E1059D7F9093E1058093E00581E0809359054DC080910A0690910B06CB
S12336C08D599F4FE4F082E08093590581E080930F0680910706809318060E9419168091B1
S12336E0DE059091DF05880F991F90938900809388008091E0059091E1059F7726C080913E
S12337000706882311F4289801C0299883E0809359052091DE053091DF0580910A06909157
S12337200B06820F931F90938900809388008091E0059091E1059F779093E1058093E005D6
S12337408091E0059091E10592609093E1058093E0055D9818C0109259058091DE05909193
S1233760DF0584529A4F90938B0080938A008091E0059091E10590689093E1058093E00561
S12337805D9A289A299A2D987894FF91EF91BF91AF919F918F917F916F915F914F913F9138
S12337A02F911F910F900FBE0F901F90189508951F920F920FB60F921124F89478940F906D
S12337C00FBE0F901F9018951F920F920FB60F92112478940F900FBE0F901F901895089520
S12337E008950895089588E98093C10083E18093C40080E696E090931E0680931D069093F2
S12338001A068093190680E296E090931C0680931B069093A1068093A00610921F06109215
S1233820DD0508951F920F920FB60F9211248F939F93EF93FF9380911F06882311F1E0915C
S12338401D06F0911E0681918093C600F0931E06E0931D06E05AF64030F080E696E09093E5
S12338601E0680931D0680911F06815080931F0680911F06882329F48091C1008F7D8093BC
S1233880C100FF91EF919F918F910F900FBE0F901F9018951F920F920FB60F9211242F93ED
S12338A08F939F93EF93FF938091C600E091A006F091A10680838091DD058F5F8093DD05AD
S12338C08091A0069091A10601969093A1068093A0068056964030F080E296E09093A106DD
S12338E08093A006FF91EF919F918F912F910F900FBE0F901F9018958091DD05882319F4D9
S12339008FEF9FEF0895F8948091DD0581508093DD05E0911B06F0911C062191F0931C0629
S1233920E0931B06E056F64030F080E296E090931C0680931B067894822F90E00895982F81
S123394080911F068F33E0F780911F06803418F080E090E00895F89480911F068F5F809372
S12339601F06E0911906F0911A0690838091190690911A06019690931A0680931906805A83
S1233980964030F080E696E090931A06809319068091C10080628093C100789481E090E077
S12339A00895CF93DF93EC0104C00E949F1C8111219688818823C9F781E090E0DF91CF9126
S12339C0089583EC94E00E94D11C08958BEC94E00E94D11C08958091DD0590E00895CF92BF
S12339E0DF92EF92FF920F931F93CF93DF93CDB7DEB729970FB6F894DEBF0FBECDBF8C016B
S1233A00F62EE42EDE011196EEECF4E089E001900D928150E1F749E06E010894C11CD11CF8
S1233A20FF2081F089E090E0841B91092F2D30E08217930738F04150F601E40FF11D8CE222
S1233A408083FF244150F601E40FF11DC8016AE070E00E94841D805D8083C8016AE070E0CA
S1233A600E94841D8B01672B11F4FF2019F085E08F15B0F619E01E197E010894E11CF11CB0
S1233A8007C0F701E10FF11D80810E949F1C1F5F1930B8F329960FB6F894DEBF0FBECDBF8F
S1233AA0DF91CF911F910F91FF90EF90DF90CF900895629FD001739FF001829FE00DF11D78
S1233AC0649FE00DF11D929FF00D839FF00D749FF00D659FF00D9927729FB00DE11DF91FE2
S1233AE0639FB00DE11DF91FBD01CF0111240895991B79E004C0991F961708F0961B881F07
S1233B007A95C9F780950895AA1BBB1B51E107C0AA1FBB1FA617B70710F0A61BB70B881F44
S1233B20991F5A95A9F780959095BC01CD01089597FB092E07260AD077FD04D0E5DF06D026
S1233B4000201AF4709561957F4F0895F6F7909581959F4F0895A1E21A2EAA1BBB1BFD01B6
S1233B600DC0AA1FBB1FEE1FFF1FA217B307E407F50720F0A21BB30BE40BF50B661F771FB7
S1233B80881F991F1A9469F760957095809590959B01AC01BD01CF01089597FB092E052618
S1233BA00ED057FD04D0D7DF0AD0001C38F450954095309521953F4F4F4F5F4F0895F6F78A
S1233BC090958095709561957F4F8F4F9F4F0895F999FECFB2BDA1BDF89A119600B40895BF
S1233BE0F7DFE02DF5DFF02D0895F999FECFB2BDA1BD00BC11960FB6F894FA9AF99A0FBE7C
S1233C000895F3DF012CF1DF11240895FFCF2F000100020003000400050006000700080041
S1233C203228E803900106141E3C401F6419121E01010203040A0411C4098813AC0D646417
S1233C4000DCE64003020A14324696500054819596B7AFC3C8BEBEB9B0AFAFADAC4984C0C3
S1233C60CBD2D6D7D0C7C2BBB8B3AEAAA9458AA2A9AAB7C0BABEBBB6B8B2B3B4B93281868F
S1233C808DA4A58B8C8F9EA6A2A6A5A6C034525D5B596F788285858281FF859FB034444E67
S1233CA04B4A54615769727272737D9095272C1B252B334B5155616A6D6C7D828B1D211A23
S1233CC0242A32454C4F5E6169717E818634323232323232323232327F323232323232325D
S1233CE032323232323232323232323232131718191B1C1D1F21232527282C2E31141819E0
S1233D001A1C2124272B3035393C3E414316191D232A31353B3F42484E565A5E651B1D3604
S1233D203E525863666C6E777D84898D932226434B6172818A9097A8ACAFB1B6B9292E4836
S1233D404E6B7C939BA2AFB9BFCBD2D2D229344B536E7F9CA8B1BCC5D0D2D2D2D2283F4EC7
S1233D60587187A4B2BAC2D2D2D2D2D2D23746545E7691B1BEC4D2D2D2D2D2D2D239485633
S1233D8060869FBAD2D2D2D2D2D2D2D2D2000000000000000000000000000000000000007E
S1233DA00000000000000000000000000000000000000000000000000000000000000000FF
S1233DC0000000000000000000000000000102030405060708090A0B0C0D0E0F1001020351
S1233DE00405060708090A0B0C0D0E0F100102030405060708090A0B0C0D0E0F1014161774
S1233E0018191A1B1C1D1E1F2021222324191A1B1C1D1E1F2021222324252627271E1F20B4
S1233E2022232425262728292A2B2C2D2E000204060708090A0C0E28262422201E1E1E1E02
S1233E401E1E1E1E1E1E1EF0FF80BBE0880465484BA438022BF0207019CC13860F440CC2D6
S1233E6009D0074C061B052A046A03D1025602F201A1015F012801FB00D600B7009D00875C
S1233E80007500660059004D0044003C0034002E0029002500F0FF80BBE0880465484BA43B
S1233EA038022BF0207019CC13860F440CC209D0074C061B052A046A03D1025602F201A1CE
S1233EC0015F012801FB00D600B7009D0087007500660059004D0044003C0034002E00291C
S1233EE0002500F0FF80BBE0880465484BA438022BF0207019CC13860F440CC209D0074CB7
S1233F00061B052A046A03D1025602F201A1015F012801FB00D600B7009D0087007500660C
S1233F200059004D0044003C0034002E0029002500F0FF80BBE0880465484BA438022BF020
S1233F40207019CC13860F440CC209D0074C061B052A046A03D1025602F201A1015F0128F9
S1233F6001FB00D600B7009D0087007500660059004D0044003C0034002E002900250000DF
S1233F8000F5047E05AE066C08C00AB30D630F8B10D7118813000000000A000F001E003CEC
S1233FA0007800FA007201E00180028002000008000A000C000E00C80A4A067E0484036F6D
S1233FC06F79797A7B7E7E7E7E7E7E7E7E7E7EF4011B5B481B5B324A000D0A00202020205F
S1093FE020202020200037
S5030200FA
